:1000000096C0BCC099C377C172C1B8C0B7C0B6C0F2
:10001000B5C0B4C0B3C0B2C070C1B0C0AFC081453C
:1000200086468B479048944997609B619E62A16386
:10003000A464A765AA66AC67AE68B069B280B481F3
:10004000B682B883BA84BB84BD84FF21040714231D
:100050003764A0FFFFFFFFFFFFFFFFFFFFFFFFFF72
:100060000000000000000000000000000000234528
:100070006C98C9FF040714233764A0FFFFFFFFFF3C
:10008000FFFFFFFFFFFFFF00000000000000000077
:1000900023405F7AB4FFFFFFFFFFFF001400081446
:1000A00000080E140004080E14000305080E1400C6
:1000B00004080A0E1114000305080A0E10140003A8
:1000C00005080A0E1012140008000E00080E0004A5
:1000D000080E000305080E0004080E1100080E119A
:1000E00000F3F404080E10121400080A0C0E0F108E
:1000F000121400080EED140002030405000414009D
:10010000040E1400040810140004080F1114000356
:1001100005080A0E0004080A0E00EEEDECEB140EC2
:1001200008040004080E00EBECEDEEF3F4141124C7
:100130001FBECFE5D1E0DEBFCDBF20E0A0E6B0E03E
:1001400001C01D92AA37B207E1F7EBE7F0E085E5C1
:10015000808781E083831482128287E08683118204
:10016000118688E58287E1E6F0E08DEF87838EEFE8
:100170008583712C55245A94C1D0F9C241CF989AE5
:100180001EBC1BBC19BC18BC089525B7277E25BF13
:1001900021E02FBD019728F020E288952150E9F752
:1001A000F9CF089588EE93E0F0CF369A3699FECFD6
:1001B00095B18091600089270895CF93C72D81E084
:1001C000870D8F73782E662D90E0C3D26FEF8C2F42
:1001D00090E0CF91BEC2FF920F931F93CF93DF9316
:1001E000F82E0CE710E0CEE7D0E0F11005C0CE010C
:1001F000A8D2F801808304C0F8016081CE01A9D2A1
:1002000021970F5F1F4FC437D10579F7DF91CF9149
:100210001F910F91FF900895D0DF81E0DCCF811115
:1002200001C0ADCF815090E0FC01E45BFF4FE49151
:10023000EEBD9898FC01E05AFF4FE491EBBDFC0144
:10024000EC58FF4FE491E9BDFC01E857FF4F849162
:1002500088BD08950F931F93CF93C82F8B01CC2394
:1002600059F085E0DCDFC80190DF89DFC8018DDF50
:10027000C8018BDFC150F3CFCF911F910F9108952B
:10028000EF92FF920F931F93CF93C8E0E82EF12CCB
:10029000062F10E084E1C3DFC70177DF70DFC801FC
:1002A00074DFC150B9F7CF911F910F91FF90EF907C
:1002B00008951F93CF93DF938FEA87B986EC86B9B1
:1002C0001092600010E1C0E0D0E085E090E05DDFDA
:1002D0006CDFC80FD11D1150C1F7CE0124E09695F7
:1002E00087952A95E1F7DF91CF911F91089598990D
:1002F00001C0C39A1895C3981895189510927A0062
:1003000087E790E01ED2853519F0612C85DF11C09A
:10031000712C872D90E015D2682E8F3F19F080E068
:100320005ADF07C0872D91E0970D792E803488F32E
:10033000F6CF20918400C0917E0010917F008091C3
:100340007C00882319F010E0C0E02AE12F5F90E0E4
:1003500040E050E0ACE9B0E0222379F0BD016F5FEE
:100360007F4FFB013197E491EE2319F0962F9A1BF2
:10037000F6CF2150AD01DB01EFCF092F6C2F70E0DC
:10038000A92FB0E0E02FF0E0112321F09D012E1BFA
:100390003F0B05C09F0121503109260F371F3197B0
:1003A000E40FF51FF49026593F4FF901F0820150F8
:1003B00049F79C0F90938600CC2371F0112329F00C
:1003C000292F30E02150310902C020E030E0F9014E
:1003D000E659FF4F41E0408327E0290F322F31508B
:1003E000E32FE91BF0E0E95DFE4FE491A32FB0E0BD
:1003F000A659BF4FEC933913F2CFE22FF0E0E75943
:10040000FF4F31E050916A004081541330E0231BCC
:1004100020938700362D353FE8F5452D4330B0F465
:10042000809188008F3F29F480917A008093880022
:1004300006C081E0860D682E891708F0612C809136
:1004400088008F5F8F718093880024C030917A007C
:10045000309388004630C0F430918100332311F08E
:10046000882339F081E0860D682E891798F0612C79
:1004700011C0862D6916D9F3662019F08150682EB7
:1004800009C02150622E06C08111F1CF80917D00FC
:10049000882369F3512C8FEF8DBD80E68CBD89B721
:1004A000846489BFAA9A8FE384BB8BE187BB80EE0B
:1004B00088BB81E083BF81EA8ABD82E480BF8BB7BD
:1004C00080628BBF8AB785608ABF85B7806285BF2F
:1004D00078948CE287B986EC86B93699FECF8FEF97
:1004E00080936000C62DC53F10F0612C3CC0809108
:1004F0008800803138F4E62DF0E0E659FF4FC081E6
:10050000DC2F31C04FDE80917A0080938800CCE7E9
:10051000D0E000E010E0FF24F39481E0800F0F5F53
:100520001F4F98819F3F29F4219608301105A9F7A4
:10053000E2CF6DE570E08EDEF801EF59FF4F60808D
:1005400088818F25888368DE6FE070E080E282DE3C
:1005500088818F258883612C5FDE24DE80917C007A
:10056000882311F3C8CF29DE10E0F12C8CE2D82EBD
:1005700096ECC92EEE24EA94CE3E19F463E481E2AF
:1005800004C0CD3E21F468E284E17ADE76C0CC3E40
:1005900011F469E203C0CB3E19F462E581E0F5CFC6
:1005A000C33F81F404E084E13ADE85E090E0EDDDD4
:1005B00088E035DE81E490E0E8DD0150A1F780EDD0
:1005C00092E05AC0C43F51F584E690E0DEDDEDDDF7
:1005D00090E0292F30E0F901E25EFF4FE491E81747
:1005E00010F49E5FF6CFF901E15EFF4F04916DE7D5
:1005F00070E0802F8295869587702CDE8EEE92E0DB
:10060000C4DD65E070E081E025DE85E694E0BDDDD7
:100610006DE770E0802F8F711DDE0DC0CE3F71F44D
:1006200000E000938400F8DD6AEF70E081E012DE04
:100630000F5F0A31B1F7B6DDB5DD1FC0CD3F69F5FB
:100640008FEF80938500E8DD85E0E9DDABDDAADD95
:1006500084E1E5DD2EDE80938500DEDDA3DDA2DD15
:10066000F9CF3699FECFE0926000F3949091850027
:100670008917C8F484EF91E088DD80917A00809337
:10068000880093DD803998F51F5F183008F474CF27
:10069000D53190F010E0DAE0CAE08D2FC0DD09DE40
:1006A000D7B8C6B8DECFDB3028F3F4E1FF1510F77A
:1006B000E0927A00DAE0DECFD23030F08D2F8695EE
:1006C0008695D695D80F12C05ADD85B7877E806192
:1006D00085BFF89485B7846885BF8B7F85BF85B754
:1006E000806285BF889585B78F7D85BFCD2F10E04F
:1006F00043CF112416B843DD87B3847E87BB94E4CF
:10070000B29914C05394999885B7877E806185BF4C
:10071000A89591BD85B7846885BF8B7F85BF789488
:100720008895F89481B58F7B81BDEACF8FE58DBF29
:1007300081E08EBF1FBEE2DD552011F0189501C08B
:10074000D8DFE199FECF1FBA8EBBE09A99278DB30F
:100750000895262FE199FECF1CBA1FBA8EBB2DBB80
:100760000FB6F894E29AE19A0FBE01960895F894B4
:02077000FFCFB9
:00000001FF
